:100000000C945A000C946C000C946C000C946C00D2
:100010000C946C000C946C000C946C000C946C00B0
:100020000C946C000C946C000C9423020C946C00E7
:100030000C946C000C946C000C946C000C946C0090
:100040000C946C000C946C000C946C000C946C0080
:100050000C946C000C946C000C946C000C946C0070
:100060000C946C000C946C000C946C000C946C0060
:100070000C946C000C946C000C946C000C946C0050
:100080000C946C000C946C000C946C000C94F203B7
:100090000C946C000C946C000C946C000C946C0030
:1000A0000C946C000C946C000C946C000C946C0020
:1000B0000C946C0011241FBECFEFD8E0DEBFCDBF83
:1000C00021E0A0E0B1E001C01D92A831B207E1F744
:1000D0000E9459020C949B040C9400008F929F92F2
:1000E000AF92BF92CF92DF92EF92FF9288E090E0C2
:1000F0000E946A046B017C0184E090E00E946A0423
:100100004B015C0180E090E00E946A0425E0C21689
:10011000D1042EEFE2062FEAF20661F475016401C4
:10012000C094D094E094F0946C157D058E059F05E5
:1001300009F450C084E593E3A5E0B0E080930001AA
:1001400090930101A0930201B09303014FEA5AEA90
:1001500064E575E088E090E00E94700488E090E03B
:100160000E942B0440910001509101016091020115
:100170007091030184E090E00E94700488E090E0B8
:100180000E942B04409100015091010160910201F5
:1001900070910301409550956095709580E090E0D6
:1001A0000E94700488E090E00E942B0445E050E03B
:1001B0006EEF7FEA88E090E00E94700488E090E0B3
:1001C000FF90EF90DF90CF90BF90AF909F908F9077
:1001D0000C942B048092000190920101A0920201E4
:1001E000B0920301FF90EF90DF90CF90BF90AF905F
:1001F0009F908F900895CF92DF92EF92FF92AC0183
:100200009C0136952795C0900001D0900101E090A7
:100210000201F0900301C701B601620F731F811D37
:10022000911D9A0140E050E00E943904C901FF90FD
:10023000EF90DF90CF900895CF92DF92EF92FF92F0
:10024000AC019C0136952795C0900001D09001012A
:10025000E0900201F0900301C701B601620F731F25
:10026000811D911D9A0140E050E00E943904C901AE
:10027000FF90EF90DF90CF9008958823A9F08091B0
:10028000000190910101A0910201B0910301805EF3
:100290009C4FAF4FBF4F8093000190930101A093FB
:1002A0000201B09303010895809100019091010132
:1002B000A0910201B091030180529340A109B109BC
:1002C0008093000190930101A0930201B093030178
:1002D00008954FEA5AEA64E575E088E090E00E94EC
:1002E000700488E090E00E942B044091000150913E
:1002F0000101609102017091030184E090E00E948D
:10030000700488E090E00E942B044091000150911D
:100310000101609102017091030140955095609533
:10032000709580E090E00E94700488E090E00E9468
:100330002B0445E050E06EEF7FEA88E090E00E94F9
:10034000700488E090E00C942B0410920E0110923F
:100350000F01109210011092110110920D011092D4
:100360000C0110920B0110920A01109209010E94D7
:100370001D049093080180930701109206011092CA
:100380000501109204012098289AE1E8F0E080E845
:10039000808380E280936F008081826080830895F3
:1003A00080910901811110C080910701909108018D
:1003B0000E9422048136910530F0109206011092BD
:1003C00005011092040108950E941D0490930801F4
:1003D000809307012091060121110EC020910C018C
:1003E00030910D0130930B0120930A0121E02093FD
:1003F000060110920901DCCF80910C0190910D0152
:1004000020910A0130910B01821B930B0E941C0169
:100410009093050180930401809107019091080158
:10042000DDCF8091040190910501089560910E0146
:1004300070910F018091100190911101089583B185
:100440008095817008951F920F920FB60F9211241C
:100450008F939F93AF93BF93729A809109018111FB
:100460000BC0809186009091870090930D0180933E
:100470000C0181E08093090180910E0190910F01A0
:10048000A0911001B09111010196A11DB11D8093A1
:100490000E0190930F01A0931001B0931101729877
:1004A000BF91AF919F918F910F900FBE0F901F90B2
:1004B00018950E945A030E9419040E946E000E941F
:1004C00067030E94A5010E941602162F0E941D04B8
:1004D0007C0103C0C83008F04FC00E941602C62F2E
:1004E000C11BC7010E942204813A910598F30E9422
:1004F0001D047C0106C00E941602862F811BC813B2
:100500003BC0C7010E942204803A9105A0F3C53088
:1005100009F471C0C73081F540E061E084E690E005
:100520000E94850324E6E22EF12C709A0E941602A6
:10053000D62E0E941D048C010E941602C62FCD19D2
:1005400011F1C8010E9422048134910520F5C430C4
:1005500098F30E94690140E061E086E990E00E9422
:10056000850380E490E00E942B0440E061E080E09D
:1005700090E00E948503FFCF0E9465030E941F0246
:100580000E94EC03FBCF0E941D048C010E942204F8
:100590008134910588F20E941D048C0106C00E94DE
:1005A0001602862F8D198C13D4CFC8010E94220405
:1005B0008097A8F3C230E9F0C33089F0C13049F622
:1005C00084E6E816F10409F471C084E6E82EF12C03
:1005D00040E061E0C7010E9485037098A6CF80E0EB
:1005E0000E943D0141E061E0C7010E9485037098CF
:1005F0009CCF81E0F5CF40E061E086E990E00E9489
:10060000850380E490E00E942B04C0E0709A0E9471
:10061000D0017098C13079F0C13098F0C230B1F794
:100620000E941102892BD1F0C1E0709A0E94D00182
:100630007098C13089F70E941102892B09F5C2E038
:10064000E5CF40E061E080E090E00E9485030E94F9
:100650001102C1E0892BD1F6C0E0D8CF0E94E3039C
:100660006B017C010E941602C616D706E806F90641
:1006700098F740E060E08CEB92E00E948503C6CFE3
:100680000E9411029C012B5F3F4FADECBCEC0E941D
:100690005B0496958795969587959695879540E006
:1006A00060E08C599F4F0E948503B0CF96E9E92EF8
:1006B000F12C8ECF87EF8093640084E380936500F4
:1006C0001EB88FE08DB978940895F894089510922B
:1006D0001401109215011092160110921701109238
:1006E000130110921201509A589A8AE090E0909368
:1006F00099008093980082E08093900088E1809335
:10070000910081E08093710008951F93CF93DF9350
:1007100020911201309113012817390799F0162FF3
:10072000EC010097A9F482E08093900088E1809327
:100730009100D0931301C09312017198DF91CF9172
:100740001F9108954423C9F3162FEC01009759F324
:100750000E94FB002091120130911301232BA1F084
:1007600020919600309197008217930728F5AC01ED
:10077000445151091123C1F020919400309195000A
:1007800042175307C8F304C01092950010929400CA
:10079000719A909397008093960082EC80939000DA
:1007A0008AE180939100C5CF20919400309195000B
:1007B0004217530718F2ECCF4091960050919700E2
:1007C00044515109D7CF6091140170911501809166
:1007D0001601909117010895882311F058980895F3
:1007E000589A08951F920F920FB60F9211248F936B
:1007F0009F93AF93BF93739A8091140190911501C9
:10080000A0911601B09117010196A11DB11D809311
:10081000140190931501A0931601B09317017398DA
:10082000BF91AF919F918F910F900FBE0F901F902E
:10083000189585E08093A10008958091A40090917F
:10084000A50008952091A4003091A500A901481B9E
:10085000590BCA0108954091A4005091A500209120
:10086000A4003091A500241B350B28173907B8F3D5
:100870000895A1E21A2EAA1BBB1BFD010DC0AA1FE1
:10088000BB1FEE1FFF1FA217B307E407F50720F0F9
:10089000A21BB30BE40BF50B661F771F881F991F74
:1008A0001A9469F760957095809590959B01AC01BD
:1008B000BD01CF010895A29FB001B39FC001A39FC6
:1008C000700D811D1124911DB29F700D811D112489
:1008D000911D0895A6E1B0E044E050E00C947F043F
:1008E000242F0E948E04252F0E948E040C947804DD
:1008F0000E948D04272F0C948E04DC01CB01FC0197
:10090000F999FECF06C0F2BDE1BDF89A319600B468
:100910000D9241505040B8F70895262FF999FECF17
:100920001FBA92BD81BD20BD0FB6F894FA9AF99A0C
:0A0930000FBE01960895F894FFCF62
:00000001FF
